 lcdc

 Timestamp is 4fb04cb9 (Mon May 14 12:07:21 2012)

 Preferred load address is 10000000

 Start         Length     Name                   Class
 0001:00000000 00000004H .CRT$XCA                CODE
 0001:00000004 00000004H .CRT$XCU                CODE
 0001:00000008 00000004H .CRT$XCZ                CODE
 0001:0000000c 00000004H .CRT$XIA                CODE
 0001:00000010 00000004H .CRT$XIZ                CODE
 0001:00000014 00000004H .CRT$XPA                CODE
 0001:00000018 00000004H .CRT$XPZ                CODE
 0001:0000001c 00000004H .CRT$XTA                CODE
 0001:00000020 00000004H .CRT$XTZ                CODE
 0001:00000030 0000172cH .rdata                  CODE
 0001:0000175c 00000021H .rdata$debug            CODE
 0001:00001780 0002184cH .text                   CODE
 0001:00022fcc 00000030H .text$yc                CODE
 0001:00022ffc 00000094H .xdata                  CODE
 0001:00023090 0000003cH .idata$2                CODE
 0001:000230cc 00000014H .idata$3                CODE
 0001:000230e0 00000154H .idata$4                CODE
 0001:00023234 000000a2H .idata$6                CODE
 0001:000232e0 0000005cH .edata                  CODE
 0002:00000000 00000154H .idata$5                DATA
 0002:00000158 0000bd70H .data                   DATA
 0002:0000bec8 00003ed4H .bss                    DATA
 0003:00000000 00000c98H .pdata                  DATA

  Address         Publics by Value              Rva+Base       Lib:Object

 0000:00000000       ___safe_se_handler_table   00000000     <absolute>
 0000:00000000       ___safe_se_handler_count   00000000     <absolute>
 0001:00000000       __xc_a                     10001000     corelib0:crt0init.obj
 0001:00000008       __xc_z                     10001008     corelib0:crt0init.obj
 0001:0000000c       __xi_a                     1000100c     corelib0:crt0init.obj
 0001:00000010       __xi_z                     10001010     corelib0:crt0init.obj
 0001:00000014       __xp_a                     10001014     corelib0:crt0init.obj
 0001:00000018       __xp_z                     10001018     corelib0:crt0init.obj
 0001:0000001c       __xt_a                     1000101c     corelib0:crt0init.obj
 0001:00000020       __xt_z                     10001020     corelib0:crt0init.obj
 0001:0000004c       ??_C@_19OBGHODPD@?$AAM?$AAo?$AAd?$AAe?$AA?$AA@ 1000104c     bsplcdc.obj
 0001:00000058       ??_C@_1CK@ENPFCICM@?$AAD?$AAr?$AAi?$AAv?$AAe?$AAr?$AAs?$AA?2?$AAD?$AAi?$AAs?$AAp?$AAl?$AAa?$AAy?$AA?2?$AAL?$AAC?$AAD?$AAC?$AA?$AA@ 10001058     bsplcdc.obj
 0001:00000084       ??_C@_1CM@JBPFNDBJ@?$AAD?$AAr?$AAi?$AAv?$AAe?$AAr?$AAs?$AA?2?$AAB?$AAu?$AAi?$AAl?$AAt?$AAI?$AAn?$AA?2?$AAL?$AAC?$AAD?$AAA?$AAD?$AA?$AA@ 10001084     bsplcdc.obj
 0001:000000b0       ??_C@_1BE@NLLCHOPM@?$AAW?$AAa?$AAl?$AAl?$AAp?$AAa?$AAp?$AAe?$AAr?$AA?$AA@ 100010b0     bsplcdc.obj
 0001:000000c4       ??_C@_1CK@NGGJLNDN@?$AAC?$AAo?$AAn?$AAt?$AAr?$AAo?$AAl?$AAP?$AAa?$AAn?$AAe?$AAl?$AA?2?$AAD?$AAe?$AAs?$AAk?$AAt?$AAo?$AAp?$AA?$AA@ 100010c4     bsplcdc.obj
 0001:000001a8       ??_7MXDDLcdc@@6B@          100011a8     lcdc_common_topaz_v1:DDLcdc.obj
 0001:00000344       ??_C@_1CG@JHDABJCF@?$AAM?$AAo?$AAu?$AAs?$AAe?$AAD?$AAe?$AAt?$AAa?$AAc?$AAh?$AAe?$AAd?$AAE?$AAv?$AAe?$AAn?$AAt?$AA?$AA@ 10001344     lcdc_common_topaz_v1:DDLcdcCursor.obj
 0001:0000036c       ??_C@_1CG@NNBNONKD@?$AAM?$AAo?$AAu?$AAs?$AAe?$AAA?$AAt?$AAt?$AAa?$AAc?$AAh?$AAe?$AAd?$AAE?$AAv?$AAe?$AAn?$AAt?$AA?$AA@ 1000136c     lcdc_common_topaz_v1:DDLcdcCursor.obj
 0001:000005c0       ??_7MXDDLcdcSurf@@6B@      100015c0     lcdc_common_topaz_v1:DDLcdcSurf.obj
 0001:00000774       ??_C@_1M@FIJHFMPA@?$AAA?$AAN?$AAG?$AAL?$AAE?$AA?$AA@ 10001774     lcdc_common_topaz_v1:DDLcdcRotate.obj
 0001:00000780       ??_C@_1CI@PNCEGBJC@?$AAS?$AAY?$AAS?$AAT?$AAE?$AAM?$AA?2?$AAG?$AAD?$AAI?$AA?2?$AAR?$AAO?$AAT?$AAA?$AAT?$AAI?$AAO?$AAN?$AA?$AA@ 10001780     lcdc_common_topaz_v1:DDLcdcRotate.obj
 0001:00000860       ??_C@_1GI@LBPPMOKF@?$AA?$HL?$AA?$CF?$AA0?$AA8?$AAl?$AAX?$AA?9?$AA?$CF?$AA0?$AA4?$AAX?$AA?9?$AA?$CF?$AA0?$AA4?$AAX?$AA?9?$AA?$CF?$AA0?$AA2?$AAX?$AA?$CF?$AA0?$AA2?$AAX?$AA?9?$AA?$CF?$AA0?$AA2?$AAX?$AA?$CF?$AA0@ 10001860     lcdc_common_topaz_v1:DDLcdcPower.obj
 0001:000008c8       ??_C@_1CE@LGAKADBG@?$AAD?$AAi?$AAs?$AAp?$AAl?$AAa?$AAy?$AAP?$AAo?$AAw?$AAe?$AAr?$AAC?$AAl?$AAa?$AAs?$AAs?$AA?$AA@ 100018c8     lcdc_common_topaz_v1:DDLcdcPower.obj
 0001:000008f0       ??_C@_1EO@BHDHHEGO@?$AA?$HL?$AAE?$AAB?$AA9?$AA1?$AAC?$AA7?$AAC?$AA9?$AA?9?$AA8?$AAB?$AAF?$AA6?$AA?9?$AA4?$AAa?$AA2?$AAd?$AA?9?$AA9?$AAA?$AAB?$AA8?$AA?9?$AA6?$AA9?$AA7?$AA2?$AA4?$AAE?$AAE@ 100018f0     lcdc_common_topaz_v1:DDLcdcPower.obj
 0001:00000940       ??_C@_1CG@BEPCNIEH@?$AAS?$AAy?$AAs?$AAt?$AAe?$AAm?$AA?2?$AAG?$AAD?$AAI?$AA?2?$AAD?$AAr?$AAi?$AAv?$AAe?$AAr?$AAs?$AA?$AA@ 10001940     lcdc_common_topaz_v1:DDLcdcPower.obj
 0001:00000c48       ?EDDGPEPixelFormatToEGPEFormat@@3QBW4EGPEFormat@@B 10001c48     ddgpe:ddgpe.obj
 0001:00000c94       ?EGPEFormatToEDDGPEPixelFormat@@3QBW4EDDGPEPixelFormat@@B 10001c94     ddgpe:ddgpe.obj
 0001:00000cc0       ??_7DDGPE@@6B@             10001cc0     ddgpe:ddgpe.obj
 0001:00000e5c       ??_7GPESurf@@6B@           10001e5c     ddgpe:ddgpesurf.obj
 0001:00000e60       ??_7DDGPESurf@@6B@         10001e60     ddgpe:ddgpesurf.obj
 0001:00000ea8       g_NullBlendFunction        10001ea8     gpe:ddi_if.obj
 0001:00000f2c       ??_C@_17BJMBELJK@?$AAG?$AAP?$AAE?$AA?$AA@ 10001f2c     gpe:ddi_if.obj
 0001:00000f34       EGPEFormatToBpp            10001f34     gpe:gpe.obj
 0001:00000f58       EGPEFormatToIFormat        10001f58     gpe:gpe.obj
 0001:00000f7c       IFormatToEGPEFormat        10001f7c     gpe:gpe.obj
 0001:00000fa8       ??_7GPE@@6B@               10001fa8     gpe:gpe.obj
 0001:00001024       ??_C@_1BM@OHJNPODK@?$AAA?$AAs?$AAp?$AAe?$AAc?$AAt?$AAR?$AAa?$AAt?$AAi?$AAo?$AAX?$AAY?$AA?$AA@ 10002024     gpe:gpe.obj
 0001:00001040       ??_C@_1BK@GPCKCPMK@?$AAA?$AAs?$AAp?$AAe?$AAc?$AAt?$AAR?$AAa?$AAt?$AAi?$AAo?$AAY?$AA?$AA@ 10002040     gpe:gpe.obj
 0001:0000105c       ??_C@_1BK@NHJGEIKP@?$AAA?$AAs?$AAp?$AAe?$AAc?$AAt?$AAR?$AAa?$AAt?$AAi?$AAo?$AAX?$AA?$AA@ 1000205c     gpe:gpe.obj
 0001:00001078       ??_C@_1BO@ONBCMHFO@?$AAL?$AAo?$AAg?$AAi?$AAc?$AAa?$AAl?$AAP?$AAi?$AAx?$AAe?$AAl?$AAs?$AAY?$AA?$AA@ 10002078     gpe:gpe.obj
 0001:00001098       ??_C@_1BO@FFKOKADL@?$AAL?$AAo?$AAg?$AAi?$AAc?$AAa?$AAl?$AAP?$AAi?$AAx?$AAe?$AAl?$AAs?$AAX?$AA?$AA@ 10002098     gpe:gpe.obj
 0001:000010b8       ??_C@_1BK@HNDINEGH@?$AAV?$AAe?$AAr?$AAt?$AAi?$AAc?$AAa?$AAl?$AAS?$AAi?$AAz?$AAe?$AA?$AA@ 100020b8     gpe:gpe.obj
 0001:000010d4       ??_C@_1BO@CPEMBNKP@?$AAH?$AAo?$AAr?$AAi?$AAz?$AAo?$AAn?$AAt?$AAa?$AAl?$AAS?$AAi?$AAz?$AAe?$AA?$AA@ 100020d4     gpe:gpe.obj
 0001:00001780       ?BSPGetFrameBuffer@@YAKXZ  10002780 f   bsplcdc.obj
 0001:0000178c       ?BSPGetModes@@YAPAUGPEMode@@XZ 1000278c f   bsplcdc.obj
 0001:000017a0       ?BSPGetModeNum@@YAKXZ      100027a0 f   bsplcdc.obj
 0001:000017a8       ?BSPGetModeDescriptor@@YAHHPAULCDC_MODE_DESCRIPTOR@@@Z 100027a8 f   bsplcdc.obj
 0001:00001814       ?BSPDeinitLCDC@@YAHPAULCDC_MODE_DESCRIPTOR@@@Z 10002814 f   bsplcdc.obj
 0001:0000181c       ?BSPPowerOnDisplay@@YAXPAULCDC_MODE_DESCRIPTOR@@@Z 1000281c f   bsplcdc.obj
 0001:00001820       ?BSPPowerOffDisplay@@YAXPAULCDC_MODE_DESCRIPTOR@@@Z 10002820 f   bsplcdc.obj
 0001:00001824       ?BSPGetVideoMemorySize@@YAKPAULCDC_MODE_DESCRIPTOR@@@Z 10002824 f   bsplcdc.obj
 0001:00001830       ?BSPGetCacheMode@@YAHXZ    10002830 f   bsplcdc.obj
 0001:000018e0       ?BSPInitLCDC@@YAHXZ        100028e0 f   bsplcdc.obj
 0001:00001ee0       ?BSPTurnOnDisplay@@YAXPAULCDC_MODE_DESCRIPTOR@@@Z 10002ee0 f   bsplcdc.obj
 0001:00001ef0       ?BSPTurnOffDisplay@@YAXPAULCDC_MODE_DESCRIPTOR@@@Z 10002ef0 f   bsplcdc.obj
 0001:00001f8c       DrvEnableDriver            10002f8c f   lcdc_common_topaz_v1:DDLcdc.obj
 0001:00001f9c       ?GetModeInfo@MXDDLcdc@@UAAJPAUGPEMode@@H@Z 10002f9c f   lcdc_common_topaz_v1:DDLcdc.obj
 0001:00001ff4       ?GetModeInfoEx@MXDDLcdc@@UAAJPAUGPEModeEx@@H@Z 10002ff4 f   lcdc_common_topaz_v1:DDLcdc.obj
 0001:00002044       ?NumModes@MXDDLcdc@@UAAHXZ 10003044 f   lcdc_common_topaz_v1:DDLcdc.obj
 0001:00002054       ?GetPhysicalVideoMemory@MXDDLcdc@@UAAXPAK0@Z 10003054 f   lcdc_common_topaz_v1:DDLcdc.obj
 0001:00002068       ?Init@MXDDLcdc@@AAAHXZ     10003068 f   lcdc_common_topaz_v1:DDLcdc.obj
 0001:0000213c       ?AllocVideoMemory@MXDDLcdc@@AAAHXZ 1000313c f   lcdc_common_topaz_v1:DDLcdc.obj
 0001:000022cc       ?FreeVideoMemory@MXDDLcdc@@AAAHXZ 100032cc f   lcdc_common_topaz_v1:DDLcdc.obj
 0001:00002340       ?SetRGBQuadPalette@MXDDLcdc@@QAAJPBUtagRGBQUAD@@GG@Z 10003340 f   lcdc_common_topaz_v1:DDLcdc.obj
 0001:000023b4       ?SetPalette@MXDDLcdc@@UAAJPBUtagPALETTEENTRY@@GG@Z 100033b4 f   lcdc_common_topaz_v1:DDLcdc.obj
 0001:00002428       ?SetModeHardware@MXDDLcdc@@AAAHH@Z 10003428 f   lcdc_common_topaz_v1:DDLcdc.obj
 0001:000026e8       ?Cleanup@MXDDLcdc@@AAAXXZ  100036e8 f   lcdc_common_topaz_v1:DDLcdc.obj
 0001:00002838       ?IntrProc@MXDDLcdc@@AAAKXZ 10003838 f   lcdc_common_topaz_v1:DDLcdc.obj
 0001:000028d0       ?MXDDLcdcIntr@@YAKPAVMXDDLcdc@@@Z 100038d0 f   lcdc_common_topaz_v1:DDLcdc.obj
 0001:000028e4       DrvGetMasks                100038e4 f   lcdc_common_topaz_v1:DDLcdc.obj
 0001:00002940       ?GetPhysicalModeId@DDGPE@@UAAKXZ 10003940 f i lcdc_common_topaz_v1:DDLcdc.obj
 0001:00002948       ?GetDriverData@DDGPE@@UAAPAUDDGPEDriverData@@XZ 10003948 f i lcdc_common_topaz_v1:DDLcdc.obj
 0001:00002950       ?SetDriverData@DDGPE@@UAAXPAUDDGPEDriverData@@@Z 10003950 f i lcdc_common_topaz_v1:DDLcdc.obj
 0001:00002958       ?GetGraphicsCaps@MXDDLcdc@@UAAKXZ 10003958 f i lcdc_common_topaz_v1:DDLcdc.obj
 0001:00002964       ?SetMode@MXDDLcdc@@UAAJHPAPAUHPALETTE__@@@Z 10003964 f   lcdc_common_topaz_v1:DDLcdc.obj
 0001:00002d90       ?ReInit@MXDDLcdc@@AAAHXZ   10003d90 f   lcdc_common_topaz_v1:DDLcdc.obj
 0001:00002eb8       ?InitHardware@MXDDLcdc@@AAAHXZ 10003eb8 f   lcdc_common_topaz_v1:DDLcdc.obj
 0001:00002fec       ??0MXDDLcdc@@QAA@PAH@Z     10003fec f   lcdc_common_topaz_v1:DDLcdc.obj
 0001:00003094       ??_EMXDDLcdc@@UAAPAXI@Z    10004094 f i lcdc_common_topaz_v1:DDLcdc.obj
 0001:00003094       ??_GMXDDLcdc@@UAAPAXI@Z    10004094 f i lcdc_common_topaz_v1:DDLcdc.obj
 0001:000030d0       GetGPE                     100040d0 f   lcdc_common_topaz_v1:DDLcdc.obj
 0001:00003158       ?CursorOn@MXDDLcdc@@QAAXXZ 10004158 f   lcdc_common_topaz_v1:DDLcdcCursor.obj
 0001:00003490       ?CursorOff@MXDDLcdc@@QAAXXZ 10004490 f   lcdc_common_topaz_v1:DDLcdcCursor.obj
 0001:00003618       ?PointerBltPrepare@MXDDLcdc@@QAAXPAUGPEBltParms@@@Z 10004618 f   lcdc_common_topaz_v1:DDLcdcCursor.obj
 0001:00003748       ?MouseNotificationsThread@MXDDLcdc@@CAKPAX@Z 10004748 f   lcdc_common_topaz_v1:DDLcdcCursor.obj
 0001:000037d4       ?StopMouseNotificationsThread@MXDDLcdc@@QAAXXZ 100047d4 f   lcdc_common_topaz_v1:DDLcdcCursor.obj
 0001:00003850       ?SetPointerShape@MXDDLcdc@@UAAJPAVGPESurf@@0HHHH@Z 10004850 f   lcdc_common_topaz_v1:DDLcdcCursor.obj
 0001:0000396c       ?MovePointer@MXDDLcdc@@UAAJHH@Z 1000496c f   lcdc_common_topaz_v1:DDLcdcCursor.obj
 0001:000039d4       ?StartMouseNotificationsThread@MXDDLcdc@@QAAHXZ 100049d4 f   lcdc_common_topaz_v1:DDLcdcCursor.obj
 0001:00003a7c       ?BltPrepare@MXDDLcdc@@UAAJPAUGPEBltParms@@@Z 10004a7c f   lcdc_common_topaz_v1:DDLcdcBlt.obj
 0001:00003ad8       ?BltComplete@MXDDLcdc@@UAAJPAUGPEBltParms@@@Z 10004ad8 f   lcdc_common_topaz_v1:DDLcdcBlt.obj
 0001:00003afc       ?WrappedEmulatedLine@MXDDLcdc@@QAAJPAUGPELineParms@@@Z 10004afc f   lcdc_common_topaz_v1:DDLcdcLine.obj
 0001:00003cf8       ?Line@MXDDLcdc@@UAAJPAUGPELineParms@@W4EGPEPhase@@@Z 10004cf8 f   lcdc_common_topaz_v1:DDLcdcLine.obj
 0001:00003d1c       ?SetVisibleSurface@MXDDLcdc@@UAAXPAVGPESurf@@H@Z 10004d1c f   lcdc_common_topaz_v1:DDLcdcSurf.obj
 0001:00003d58       ?AllocSurface@MXDDLcdc@@UAAJPAPAVGPESurf@@HHW4EGPEFormat@@H@Z 10004d58 f   lcdc_common_topaz_v1:DDLcdcSurf.obj
 0001:00003d9c       ?Flip@MXDDLcdc@@QAAKPAU_DDHAL_FLIPDATA@@@Z 10004d9c f   lcdc_common_topaz_v1:DDLcdcSurf.obj
 0001:00003e64       ??0MXDDLcdcSurf@@QAA@HHKPAXHW4EGPEFormat@@W4EDDGPEPixelFormat@@PAVSurfaceHeap@@@Z 10004e64 f   lcdc_common_topaz_v1:DDLcdcSurf.obj
 0001:00003ec4       ?GetDriverData@DDGPESurf@@UAAPAUDDGPEDriverData@@XZ 10004ec4 f i lcdc_common_topaz_v1:DDLcdcSurf.obj
 0001:00003ecc       ?SetDriverData@DDGPESurf@@UAAXPAUDDGPEDriverData@@@Z 10004ecc f i lcdc_common_topaz_v1:DDLcdcSurf.obj
 0001:00003ed4       ?SurfaceSize@DDGPESurf@@UAAHXZ 10004ed4 f i lcdc_common_topaz_v1:DDLcdcSurf.obj
 0001:00003edc       ?AllocSurface@MXDDLcdc@@UAAJPAPAVDDGPESurf@@HHW4EGPEFormat@@W4EDDGPEPixelFormat@@H@Z 10004edc f   lcdc_common_topaz_v1:DDLcdcSurf.obj
 0001:00004084       ??_GMXDDLcdcSurf@@UAAPAXI@Z 10005084 f i lcdc_common_topaz_v1:DDLcdcSurf.obj
 0001:00004084       ??_EMXDDLcdcSurf@@UAAPAXI@Z 10005084 f i lcdc_common_topaz_v1:DDLcdcSurf.obj
 0001:000040c4       ?DrvEscape@MXDDLcdc@@UAAKPAU_SURFOBJ@@KKPAXK1@Z 100050c4 f   lcdc_common_topaz_v1:DDLcdcMisc.obj
 0001:00004438       ?IsBusy@MXDDLcdc@@UAAHXZ   10005438 f   lcdc_common_topaz_v1:DDLcdcMisc.obj
 0001:00004488       ?InVBlank@MXDDLcdc@@UAAHXZ 10005488 f   lcdc_common_topaz_v1:DDLcdcMisc.obj
 0001:000044b4       ?WaitForNotBusy@MXDDLcdc@@UAAXXZ 100054b4 f   lcdc_common_topaz_v1:DDLcdcMisc.obj
 0001:00004510       ?GetRotateModeFromReg@MXDDLcdc@@QAAHXZ 10005510 f   lcdc_common_topaz_v1:DDLcdcRotate.obj
 0001:000045ec       ?SetRotateParams@MXDDLcdc@@QAAXXZ 100055ec f   lcdc_common_topaz_v1:DDLcdcRotate.obj
 0001:0000462c       ?DynRotate@MXDDLcdc@@QAAJH@Z 1000562c f   lcdc_common_topaz_v1:DDLcdcRotate.obj
 0001:00004690       ?SetDisplayPower@MXDDLcdc@@AAAXW4_CEDEVICE_POWER_STATE@@@Z 10005690 f   lcdc_common_topaz_v1:DDLcdcPower.obj
 0001:0000477c       ?ConvertStringToGuid@MXDDLcdc@@AAAHPBGPAU_GUID@@@Z 1000577c f   lcdc_common_topaz_v1:DDLcdcPower.obj
 0001:00004864       ?AdvertisePowerInterface@MXDDLcdc@@AAAHPAUHINSTANCE__@@@Z 10005864 f   lcdc_common_topaz_v1:DDLcdcPower.obj
 0001:00004990       ?DisableOverlay@MXDDLcdc@@QAAJXZ 10005990 f   lcdc_common_topaz_v1:DDLcdcOverlay.obj
 0001:000049ec       ?IsOverlaySurfEqual@@YAHPAUoverlaySurf@@0@Z 100059ec f   lcdc_common_topaz_v1:DDLcdcOverlay.obj
 0001:00004aa4       ?SetOverlayPosition@MXDDLcdc@@QAAKPAU_DDHAL_SETOVERLAYPOSITIONDATA@@@Z 10005aa4 f   lcdc_common_topaz_v1:DDLcdcOverlay.obj
 0001:00004c00       ?SetVisibleSurfaceOverlay@MXDDLcdc@@QAAXPAVDDGPESurf@@@Z 10005c00 f   lcdc_common_topaz_v1:DDLcdcOverlay.obj
 0001:00004c80       ?EnableOverlay@MXDDLcdc@@QAAJXZ 10005c80 f   lcdc_common_topaz_v1:DDLcdcOverlay.obj
 0001:00004e28       ?UpdateOverlay@MXDDLcdc@@QAAKPAU_DDHAL_UPDATEOVERLAYDATA@@@Z 10005e28 f   lcdc_common_topaz_v1:DDLcdcOverlay.obj
 0001:00005190       ?LcdcVMSetAttributeEx@@YAHPAULcdcVMSetAttributeExDataStruct@@@Z 10006190 f   lcdc_common_topaz_v1:DDLcdcEscape.obj
 0001:000051e4       ?LCDCGetBaseRegAddr@@YAIXZ 100061e4 f   lcdc_mx25_topaz_v1:lcdc_base.obj
 0001:000051f0       ?LCDCGetIRQ@@YAKXZ         100061f0 f   lcdc_mx25_topaz_v1:lcdc_base.obj
 0001:000051f8       ?LCDCEnableClock@@YAHH@Z   100061f8 f   lcdc_mx25_topaz_v1:lcdc_base.obj
 0001:00005278       ?LCDCGetRefClk@@YAKPAULCDC_MODE_DESCRIPTOR@@@Z 10006278 f   lcdc_mx25_topaz_v1:lcdc_base.obj
 0001:00005340       HALInit                    10006340 f   ddgpe:ddhinit.obj
 0001:00005364       ??0SurfaceHeap@@QAA@KKPAV0@0@Z 10006364 f   ddgpe:surfheap.obj
 0001:00005394       ??1SurfaceHeap@@QAA@XZ     10006394 f   ddgpe:surfheap.obj
 0001:00005444       ?Alloc@SurfaceHeap@@QAAPAV1@K@Z 10006444 f   ddgpe:surfheap.obj
 0001:00005500       ?Free@SurfaceHeap@@QAAXXZ  10006500 f   ddgpe:surfheap.obj
 0001:00005568       ?FourCCLookup@@YAPBU_FourCCDescription@@K@Z 10006568 f i ddgpe:ddgpe.obj
 0001:000055b4       ?GetDDGPE@@YAPAVDDGPE@@XZ  100065b4 f   ddgpe:ddgpe.obj
 0001:000055c4       ??0DDGPE@@QAA@XZ           100065c4 f   ddgpe:ddgpe.obj
 0001:000055f8       ??1DDGPE@@UAA@XZ           100065f8 f   ddgpe:ddgpe.obj
 0001:00005618       ?AllocSurface@DDGPE@@UAAJPAPAVDDGPESurf@@HHW4EGPEFormat@@W4EDDGPEPixelFormat@@H@Z 10006618 f   ddgpe:ddgpe.obj
 0001:0000564c       ?AllocSurface@DDGPE@@UAAJPAPAVDDGPESurf@@PAUDDGPEAllocSurfaceData@@@Z 1000664c f   ddgpe:ddgpe.obj
 0001:000056a0       ?AllocVideoSurface@DDGPE@@UAAJPAPAVDDGPESurf@@HHW4EGPEFormat@@W4EDDGPEPixelFormat@@PAK@Z 100066a0 f   ddgpe:ddgpe.obj
 0001:00005708       ?AllocVideoSurface@DDGPE@@UAAJPAU_DDRAWI_DDRAWSURFACE_LCL@@HHW4EGPEFormat@@W4EDDGPEPixelFormat@@PAK@Z 10006708 f   ddgpe:ddgpe.obj
 0001:0000576c       ?AllocVideoSurface@DDGPE@@UAAJPAPAVDDGPESurf@@PAUDDGPEAllocSurfaceData@@PAK@Z 1000676c f   ddgpe:ddgpe.obj
 0001:000057ec       ?AllocVideoSurface@DDGPE@@UAAJPAU_DDRAWI_DDRAWSURFACE_LCL@@PAUDDGPEAllocSurfaceData@@PAK@Z 100067ec f   ddgpe:ddgpe.obj
 0001:00005838       ?AllocBackBuffer@DDGPE@@UAAJPAU_DDRAWI_DDRAWSURFACE_LCL@@@Z 10006838 f   ddgpe:ddgpe.obj
 0001:000058d4       ?WrapSurface@DDGPE@@UAAJPAU_DDRAWI_DDRAWSURFACE_LCL@@HHW4EGPEFormat@@W4EDDGPEPixelFormat@@HH@Z 100068d4 f   ddgpe:ddgpe.obj
 0001:00005944       ?WrapSurface@DDGPE@@UAAJPAPAVDDGPESurf@@HHW4EGPEFormat@@W4EDDGPEPixelFormat@@PAEH@Z 10006944 f   ddgpe:ddgpe.obj
 0001:000059b8       ?WrapSurface@DDGPE@@UAAJPAU_DDRAWI_DDRAWSURFACE_LCL@@HHW4EGPEFormat@@W4EDDGPEPixelFormat@@PAEH@Z 100069b8 f   ddgpe:ddgpe.obj
 0001:00005a24       ?WrapSurface@DDGPE@@UAAJPAPAVDDGPESurf@@PAUDDGPEAllocSurfaceData@@@Z 10006a24 f   ddgpe:ddgpe.obj
 0001:00005aa4       ?WrapSurface@DDGPE@@UAAJPAU_DDRAWI_DDRAWSURFACE_LCL@@PAUDDGPEAllocSurfaceData@@@Z 10006aa4 f   ddgpe:ddgpe.obj
 0001:00005af0       ?BltPrepare@DDGPE@@UAAJPAUDDGPEBltParms@@@Z 10006af0 f   ddgpe:ddgpe.obj
 0001:00005b80       ?PerformBlt@DDGPE@@UAAJPAUDDGPEBltParms@@@Z 10006b80 f   ddgpe:ddgpe.obj
 0001:00005bf4       ?BltExpanded@DDGPE@@UAAJPAVDDGPESurf@@000PAU_CLIPOBJ@@PAU_XLATEOBJ@@PBUtagRECT@@3KKK@Z 10006bf4 f   ddgpe:ddgpe.obj
 0001:00005d68       ?BltExpanded@DDGPE@@UAAJPAVDDGPESurf@@00PBUtagRECT@@1KKK@Z 10006d68 f   ddgpe:ddgpe.obj
 0001:00005dc4       ?SetVisibleSurface@DDGPE@@UAAXPAVGPESurf@@KH@Z 10006dc4 f   ddgpe:ddgpe.obj
 0001:00005de4       ?SetVisibleSurface@DDGPE@@UAAXPAVGPESurf@@H@Z 10006de4 f   ddgpe:ddgpe.obj
 0001:00005e44       ?DetectPixelFormat@DDGPE@@UAAJKPAU_DDPIXELFORMAT@@PAW4EGPEFormat@@PAW4EDDGPEPixelFormat@@@Z 10006e44 f   ddgpe:ddgpe.obj
 0001:000060d0       ?DetectMode@DDGPE@@UAAJPAKKKW4EGPEFormat@@W4EDDGPEPixelFormat@@PAU_DDPIXELFORMAT@@@Z 100070d0 f   ddgpe:ddgpe.obj
 0001:000061d4       ?InDisplay@DDGPE@@UAAHXZ   100071d4 f   ddgpe:ddgpe.obj
 0001:000061dc       ?GetModeInfoEx@DDGPE@@UAAJPAUGPEModeEx@@H@Z 100071dc f   ddgpe:ddgpe.obj
 0001:000061e8       ?SetMode@DDGPE@@UAAJHPAPAUHPALETTE__@@H@Z 100071e8 f   ddgpe:ddgpe.obj
 0001:000061f4       ?RegisterDDHALAPI@@YAXXZ   100071f4 f   ddgpe:ddgpe.obj
 0001:000061f8       ??_GDDGPE@@UAAPAXI@Z       100071f8 f i ddgpe:ddgpe.obj
 0001:000061f8       ??_EDDGPE@@UAAPAXI@Z       100071f8 f i ddgpe:ddgpe.obj
 0001:0000622c       ??0GPESurf@@QAA@HHPAXHW4EGPEFormat@@@Z 1000722c f i ddgpe:ddgpesurf.obj
 0001:00006284       ??_EGPESurf@@UAAPAXI@Z     10007284 f i ddgpe:ddgpesurf.obj
 0001:00006284       ??_GGPESurf@@UAAPAXI@Z     10007284 f i ddgpe:ddgpesurf.obj
 0001:000062ac       ??0DDGPESurf@@QAA@HHPAXHW4EGPEFormat@@W4EDDGPEPixelFormat@@@Z 100072ac f   ddgpe:ddgpesurf.obj
 0001:00006314       ??1DDGPESurf@@UAA@XZ       10007314 f   ddgpe:ddgpesurf.obj
 0001:0000635c       ?Init@DDGPESurf@@UAAXHHPAXHW4EGPEFormat@@W4EDDGPEPixelFormat@@@Z 1000735c f   ddgpe:ddgpesurf.obj
 0001:000063bc       ?Bpp@DDGPESurf@@UAAKXZ     100073bc f   ddgpe:ddgpesurf.obj
 0001:000063d0       ?AlignedWidth@DDGPESurf@@UAAKXZ 100073d0 f   ddgpe:ddgpesurf.obj
 0001:0000640c       ?SetColorKey@DDGPESurf@@UAAXK@Z 1000740c f   ddgpe:ddgpesurf.obj
 0001:00006448       ?ColorKey@DDGPESurf@@UAAKXZ 10007448 f   ddgpe:ddgpesurf.obj
 0001:00006464       ?SetColorKeyMask@DDGPESurf@@UAAXK@Z 10007464 f   ddgpe:ddgpesurf.obj
 0001:0000646c       ?ColorKeyMask@DDGPESurf@@UAAKXZ 1000746c f   ddgpe:ddgpesurf.obj
 0001:00006474       ?SetColorKeyLow@DDGPESurf@@UAAXK@Z 10007474 f   ddgpe:ddgpesurf.obj
 0001:0000647c       ?ColorKeyLow@DDGPESurf@@UAAKXZ 1000747c f   ddgpe:ddgpesurf.obj
 0001:00006484       ?SetColorKeyHigh@DDGPESurf@@UAAXK@Z 10007484 f   ddgpe:ddgpesurf.obj
 0001:0000648c       ?ColorKeyHigh@DDGPESurf@@UAAKXZ 1000748c f   ddgpe:ddgpesurf.obj
 0001:00006494       ?PixelFormat@DDGPESurf@@UAA?AW4EDDGPEPixelFormat@@XZ 10007494 f   ddgpe:ddgpesurf.obj
 0001:0000649c       ?HasAlpha@DDGPESurf@@UAAHXZ 1000749c f   ddgpe:ddgpesurf.obj
 0001:000064c0       ?SetDDGPESurf@DDGPESurf@@UAAXPAU_DDRAWI_DDRAWSURFACE_LCL@@@Z 100074c0 f   ddgpe:ddgpesurf.obj
 0001:000064cc       ?GetDDGPESurf@DDGPESurf@@SAPAV1@PAU_DDRAWI_DDRAWSURFACE_LCL@@@Z 100074cc f   ddgpe:ddgpesurf.obj
 0001:000064dc       ?SetRotation@DDGPESurf@@QAAXHHH@Z 100074dc f   ddgpe:ddgpesurf.obj
 0001:00006520       ??_EDDGPESurf@@UAAPAXI@Z   10007520 f i ddgpe:ddgpesurf.obj
 0001:00006520       ??_GDDGPESurf@@UAAPAXI@Z   10007520 f i ddgpe:ddgpesurf.obj
 0001:00006548       ??0DDGPESurf@@QAA@HHHW4EGPEFormat@@W4EDDGPEPixelFormat@@@Z 10007548 f   ddgpe:ddgpesurf.obj
 0001:00006620       ?DeleteSurface@DDGPESurf@@SAXPAU_DDRAWI_DDRAWSURFACE_LCL@@@Z 10007620 f   ddgpe:ddgpesurf.obj
 0001:0000664c       DllMain                    1000764c f   gpe:ddi_if.obj
 0001:00006688       ?SafeGetGPE@@YAPAVGPE@@PAX@Z 10007688 f   gpe:ddi_if.obj
 0001:000066f4       ?SetSurfaceFormat@@YAXPAVGPESurf@@PAU_XLATEOBJ@@K@Z 100076f4 f   gpe:ddi_if.obj
 0001:0000694c       DrvContrastControl         1000794c f   gpe:ddi_if.obj
 0001:00006970       DrvPowerHandler            10007970 f   gpe:ddi_if.obj
 0001:00006998       DrvEscape                  10007998 f   gpe:ddi_if.obj
 0001:00006ae0       DrvDisableDriver           10007ae0 f   gpe:ddi_if.obj
 0001:00006b10       DrvDisablePDEV             10007b10 f   gpe:ddi_if.obj
 0001:00006b3c       DrvDisableSurface          10007b3c f   gpe:ddi_if.obj
 0001:00006b60       DrvEnableSurface           10007b60 f   gpe:ddi_if.obj
 0001:00006ba4       DrvCreateDeviceBitmap      10007ba4 f   gpe:ddi_if.obj
 0001:00006c40       DrvDeleteDeviceBitmap      10007c40 f   gpe:ddi_if.obj
 0001:00006c80       DrvMovePointer             10007c80 f   gpe:ddi_if.obj
 0001:00006ca0       DrvSetPointerShape         10007ca0 f   gpe:ddi_if.obj
 0001:00006db4       DrvSetPalette              10007db4 f   gpe:ddi_if.obj
 0001:00006e40       DrvFillPath                10007e40 f   gpe:ddi_if.obj
 0001:000071fc       DrvRealizeBrush            100081fc f   gpe:ddi_if.obj
 0001:00007474       DrvGetModes                10008474 f   gpe:ddi_if.obj
 0001:00007578       DrvEnablePDEV              10008578 f   gpe:ddi_if.obj
 0001:000078ac       DrvCopyBits                100088ac f   gpe:ddi_if.obj
 0001:000078bc       ?ClipBlt@@YAJPAVGPE@@PAUGPEBltParms@@@Z 100088bc f   gpe:ddi_if.obj
 0001:00007b20       ?AAGetMaskBits@@YAXPAK00@Z 10008b20 f   gpe:ddi_if.obj
 0001:00007b60       ?GPEEnableDriver@@YAHKKPAUtagDrvEnableData@@PAU_ENGCALLBACKS@@@Z 10008b60 f   gpe:ddi_if.obj
 0001:00007c94       AnyBlt                     10008c94 f   gpe:ddi_if.obj
 0001:000084c8       DrvAnyBlt                  100094c8 f   gpe:ddi_if.obj
 0001:0000853c       DrvTransparentBlt          1000953c f   gpe:ddi_if.obj
 0001:000085bc       DrvBitBlt                  100095bc f   gpe:ddi_if.obj
 0001:000086a0       DrvPaint                   100096a0 f   gpe:ddi_if.obj
 0001:00008710       ??0GPE@@QAA@XZ             10009710 f   gpe:gpe.obj
 0001:00008758       ??1GPE@@UAA@XZ             10009758 f   gpe:gpe.obj
 0001:00008768       ?ContrastControl@GPE@@UAAHKPAK@Z 10009768 f   gpe:gpe.obj
 0001:00008770       ?PowerHandler@GPE@@UAAXH@Z 10009770 f   gpe:gpe.obj
 0001:00008774       ?GetPalette@GPE@@UAAJPAPAUtagPALETTEENTRY@@PAG@Z 10009774 f   gpe:gpe.obj
 0001:000087bc       ?DrvEscape@GPE@@UAAKPAU_SURFOBJ@@KKPAXK1@Z 100097bc f   gpe:gpe.obj
 0001:000087c4       ?GetGraphicsCaps@GPE@@UAAKXZ 100097c4 f   gpe:gpe.obj
 0001:000087cc       ?GetPhysicalVideoMemory@GPE@@UAAXPAK0@Z 100097cc f   gpe:gpe.obj
 0001:000087d0       ?SetVisibleSurface@GPE@@UAAXPAVGPESurf@@@Z 100097d0 f   gpe:gpe.obj
 0001:000087d4       ?FlipInProgress@GPE@@UAAHXZ 100097d4 f   gpe:gpe.obj
 0001:000087dc       ?WaitForVBlank@GPE@@UAAXXZ 100097dc f   gpe:gpe.obj
 0001:000087e0       ?SurfaceBusyFlipping@GPE@@UAAHPAVGPESurf@@@Z 100097e0 f   gpe:gpe.obj
 0001:000087e8       ?IsBusy@GPE@@UAAHXZ        100097e8 f   gpe:gpe.obj
 0001:000087f0       ?WaitForNotBusy@GPE@@UAAXXZ 100097f0 f   gpe:gpe.obj
 0001:000087f4       ?AvailableVideoMemory@GPE@@UAAKXZ 100097f4 f   gpe:gpe.obj
 0001:000087fc       ?ScanLine@GPE@@UAAHXZ      100097fc f   gpe:gpe.obj
 0001:00008804       ?ProcessCommandBlock@GPE@@UAAJPAE@Z 10009804 f   gpe:gpe.obj
 0001:00008810       ?GetScreenDimensions@GPE@@UAAHPAUGPEScreenProps@@@Z 10009810 f   gpe:gpe.obj
 0001:00008a58       ?IsPaletteSettable@GPE@@UAAHXZ 10009a58 f   gpe:gpe.obj
 0001:00008a70       ?RotateRectl@GPE@@QAAXPAU_RECTL@@@Z 10009a70 f   gpe:gpe.obj
 0001:00008b20       ?GetClearTypeRGBMasks@GPE@@UAAPAKXZ 10009b20 f   gpe:gpe.obj
 0001:00008b30       ?DisablePrimary@GPE@@UAAHXZ 10009b30 f   gpe:gpe.obj
 0001:00008b6c       ?Init@GPESurf@@QAAXHHPAXHW4EGPEFormat@@@Z 10009b6c f   gpe:gpe.obj
 0001:00008bc4       ?RotateLineParms@GPESurf@@QAAXPAUGPELineParms@@@Z 10009bc4 f   gpe:gpe.obj
 0001:00008c90       ?SetRotation@GPESurf@@QAAXHHH@Z 10009c90 f   gpe:gpe.obj
 0001:00008cb8       ?RotateRectl@GPESurf@@QAAXPAU_RECTL@@@Z 10009cb8 f   gpe:gpe.obj
 0001:00008d68       ?RotateRectlBack@GPESurf@@QAAXPAU_RECTL@@@Z 10009d68 f   gpe:gpe.obj
 0001:00008e20       ?GetPtr@GPESurf@@QAAPAEHH@Z 10009e20 f   gpe:gpe.obj
 0001:00008efc       ??1GPEFormat@@QAA@XZ       10009efc f   gpe:gpe.obj
 0001:00008f30       ??_GGPE@@UAAPAXI@Z         10009f30 f i gpe:gpe.obj
 0001:00008f30       ??_EGPE@@UAAPAXI@Z         10009f30 f i gpe:gpe.obj
 0001:00008f58       ??1GPESurf@@UAA@XZ         10009f58 f   gpe:gpe.obj
 0001:00008f94       ?EmulatedBlt_Internal@GPE@@QAAJPAUGPEBltParms@@@Z 10009f94 f   gpe:swblt.obj
 0001:0000b1ac       ?EmulatedBlt_Bilinear@GPE@@QAAJPAUGPEBltParms@@@Z 1000c1ac f   gpe:swblt.obj
 0001:0000ba3c       ?EmulatedBlt_Halftone@GPE@@QAAJPAUGPEBltParms@@@Z 1000ca3c f   gpe:swblt.obj
 0001:0000c2e0       ?EmulatedBltRotate_Internal@GPE@@QAAJPAUGPEBltParms@@@Z 1000d2e0 f   gpe:swblt.obj
 0001:0000efb8       ?EmulatedBltRotate_Bilinear@GPE@@QAAJPAUGPEBltParms@@@Z 1000ffb8 f   gpe:swblt.obj
 0001:0000fe74       ?EmulatedBltRotate_Halftone@GPE@@QAAJPAUGPEBltParms@@@Z 10010e74 f   gpe:swblt.obj
 0001:00010b64       ?SelectBlt@GPE@@IAAJPAUGPEBltParms@@P81@AAJ0@Z@Z 10011b64 f   gpe:swblt.obj
 0001:00010f4c       ?EmulatedBlt@GPE@@QAAJPAUGPEBltParms@@@Z 10011f4c f   gpe:swblt.obj
 0001:00010f64       ?EmulatedBltRotate@GPE@@QAAJPAUGPEBltParms@@@Z 10011f64 f   gpe:swblt.obj
 0001:00010f7c       ?EmulatedLine@GPE@@QAAJPAUGPELineParms@@@Z 10011f7c f   gpe:swline.obj
 0001:0001162c       ?Init@LRU@@QAAHG@Z         1001262c f   gpe:swconvrt.obj
 0001:000116f8       ?Find@LRU@@QAAFK@Z         100126f8 f   gpe:swconvrt.obj
 0001:000117d0       ?Add@LRU@@QAAFK@Z          100127d0 f   gpe:swconvrt.obj
 0001:00011830       ?Free@LRU@@QAAXXZ          10012830 f   gpe:swconvrt.obj
 0001:0001188c       ?InitMaskInfo@MaskInfo@@QAAXPAU_XLATEOBJ@@KG@Z 1001288c f   gpe:swconvrt.obj
 0001:00011960       ?Init@MaskColorConverter@@QAAXPAU_XLATEOBJ@@@Z 10012960 f   gpe:swconvrt.obj
 0001:00011994       ?Init@GroupColorConverter@@QAAXPAU_XLATEOBJ@@@Z 10012994 f   gpe:swconvrt.obj
 0001:00011bc8       ?RGBToFromBGR@MaskColorConverter@@QAAKK@Z 10012bc8 f   gpe:swconvrt.obj
 0001:00011c00       ?MaskedSrcToRGB@MaskColorConverter@@QAAKK@Z 10012c00 f   gpe:swconvrt.obj
 0001:00011c70       ?MaskedSrcToRGB@GroupColorConverter@@QAAKK@Z 10012c70 f   gpe:swconvrt.obj
 0001:00011ce0       ?MaskedSrcToBGR@MaskColorConverter@@QAAKK@Z 10012ce0 f   gpe:swconvrt.obj
 0001:00011d50       ?RGBSrcToMaskedDst@MaskColorConverter@@QAAKK@Z 10012d50 f   gpe:swconvrt.obj
 0001:00011d94       ?BGRSrcToMaskedDst@MaskColorConverter@@QAAKK@Z 10012d94 f   gpe:swconvrt.obj
 0001:00011dd8       ?MaskedSrcToMaskedDst@MaskColorConverter@@QAAKK@Z 10012dd8 f   gpe:swconvrt.obj
 0001:00011e58       ?AnyToMono@MonoColorConverter@@QAAKK@Z 10012e58 f   gpe:swconvrt.obj
 0001:00011e6c       DrvRealizeColor            10012e6c f   gpe:swconvrt.obj
 0001:00011fe0       DrvUnrealizeColor          10012fe0 f   gpe:swconvrt.obj
 0001:000120ec       ?Init@LookupColorConverter@@QAAXPAU_XLATEOBJ@@@Z 100130ec f   gpe:swconvrt.obj
 0001:000122d0       ?MaskedSrcToPaletteDst@GroupColorConverter@@QAAKK@Z 100132d0 f   gpe:swconvrt.obj
 0001:00012480       ?AllocConverters@@YAHXZ    10013480 f   gpe:swconvrt.obj
 0001:00012530       ?FreeConverters@@YAXXZ     10013530 f   gpe:swconvrt.obj
 0001:00012590       ?InitConverter@ColorConverter@@SAXPAU_XLATEOBJ@@PAPAV1@PAP81@AAKK@ZPAPAK@Z 10013590 f   gpe:swconvrt.obj
 0001:000127e0       ?SafeCallLine@@YAJPAVGPE@@PAUGPELineParms@@@Z 100137e0 f   gpe:drvstrok.obj
 0001:00012830       DrvStrokePath              10013830 f   gpe:drvstrok.obj
 0001:00013174       ?AATextBltInit@@YAHP6AXPAK00@Z@Z 10014174 f   gpe:aablt.obj
 0001:0001318c       ?AATextBltDst8@AATextBlt@@QAAJPAUGPEBltParms@@@Z 1001418c f   gpe:aablt.obj
 0001:00013338       ?SetGamma@AAMASKINFO@@QAAXM@Z 10014338 f i gpe:aablt.obj
 0001:00013538       ?BlendPixelAA@AAMASKINFO@@QAAKKE@Z 10014538 f   gpe:aablt.obj
 0001:000138a4       ?SetAAGammaValue@@YAHKH@Z  100148a4 f   gpe:aablt.obj
 0001:000139c4       ?AATextBltDst16@AATextBlt@@QAAJPAUGPEBltParms@@@Z 100149c4 f   gpe:aablt.obj
 0001:00013bf4       ?AATextBltDst24@AATextBlt@@QAAJPAUGPEBltParms@@@Z 10014bf4 f   gpe:aablt.obj
 0001:00013e44       ?AATextBltDst32@AATextBlt@@QAAJPAUGPEBltParms@@@Z 10014e44 f   gpe:aablt.obj
 0001:0001406c       ?AATextBltSelect@@YAJPAUGPEBltParms@@@Z 1001506c f   gpe:aablt.obj
 0001:000141bc       ?vClearTypeLookupTableLoop@@YAXKPAU_BLENDINFO@@KKPAVGPESurf@@@Z 100151bc f   gpe:rctblt.obj
 0001:00014588       ?ulBlendPixelCT@@YAKPAU_BLENDINFO@@KPAU_F_RGB@@@Z 10015588 f   gpe:rctblt.obj
 0001:000146c4       ?ulBlendPixelCT8bpp@@YAKPAU_BLENDINFO@@KPAU_F_RGB@@@Z 100156c4 f   gpe:rctblt.obj
 0001:000147a0       ?SetClearTypeBltMasks@@YAXKKK@Z 100157a0 f   gpe:rctblt.obj
 0001:0001487c       ?SetClearTypeBltGamma@@YAXK@Z 1001587c f   gpe:rctblt.obj
 0001:00014a3c       ?GetGammaValue@@YAHPAK@Z   10015a3c f   gpe:rctblt.obj
 0001:00014a58       ?SetGammaValue@@YAHKH@Z    10015a58 f   gpe:rctblt.obj
 0001:00014bfc       ?pvFillOpaqTableCT@@YAPAXKKKPAVGPESurf@@PAU_BLENDINFO@@@Z 10015bfc f   gpe:rctblt.obj
 0001:00014cb8       ?ClearTypeBltInit@@YAHPAUGPEMode@@PAKPAUtagPALETTEENTRY@@I@Z 10015cb8 f   gpe:rctblt.obj
 0001:00014e14       ?ClearTypeBltDst16@ClearTypeBlt@@QAAJPAUGPEBltParms@@@Z 10015e14 f   gpe:rctblt.obj
 0001:00014ff4       ?ClearTypeBltDst24@ClearTypeBlt@@QAAJPAUGPEBltParms@@@Z 10015ff4 f   gpe:rctblt.obj
 0001:000151ec       ?ClearTypeBltDst32@ClearTypeBlt@@QAAJPAUGPEBltParms@@@Z 100161ec f   gpe:rctblt.obj
 0001:000153cc       ?ClearTypeBltDst8@ClearTypeBlt@@QAAJPAUGPEBltParms@@@Z 100163cc f   gpe:rctblt.obj
 0001:0001559c       ?ClearTypeBltSelect@@YAJPAUGPEBltParms@@@Z 1001659c f   gpe:rctblt.obj
 0001:00015638       ??0TmpGPESurf@@QAA@PAU_SURFOBJ@@0PAV0@@Z 10016638 f   gpe:TmpGPESurf.obj
 0001:000156fc       ??0EdgeList@@QAA@H@Z       100166fc f   gpe:swfill.obj
 0001:00015744       ??1EdgeList@@QAA@XZ        10016744 f   gpe:swfill.obj
 0001:00015760       ?AddEdge@EdgeList@@QAAJJJJJ@Z 10016760 f   gpe:swfill.obj
 0001:00015994       ?Fill@EdgeList@@QAAJPAUGPEBltParms@@PAU_RECTL@@PAVGPE@@@Z 10016994 f   gpe:swfill.obj
 0001:00015e34       ?drvRectFill32@@YAXPAVGPESurf@@PAU_DRVGRADIENTRECTDATA@@@Z 10016e34 f   gpe:rdrvgradfill.obj
 0001:00016574       ?drvRectFill24@@YAXPAVGPESurf@@PAU_DRVGRADIENTRECTDATA@@@Z 10017574 f   gpe:rdrvgradfill.obj
 0001:00016bb4       ?drvRectFill16@@YAXPAVGPESurf@@PAU_DRVGRADIENTRECTDATA@@H@Z 10017bb4 f   gpe:rdrvgradfill.obj
 0001:000170ac       ?drvRectFill16_565@@YAXPAVGPESurf@@PAU_DRVGRADIENTRECTDATA@@@Z 100180ac f   gpe:rdrvgradfill.obj
 0001:000170c0       ?drvRectFill16_555@@YAXPAVGPESurf@@PAU_DRVGRADIENTRECTDATA@@@Z 100180c0 f   gpe:rdrvgradfill.obj
 0001:00017118       ?drvRectFill16Bitfields@@YAXPAVGPESurf@@PAU_DRVGRADIENTRECTDATA@@@Z 10018118 f   gpe:rdrvgradfill.obj
 0001:0001712c       ?drvRectFillPalIndex@@YAXPAVGPESurf@@PAU_DRVGRADIENTRECTDATA@@H@Z 1001812c f   gpe:rdrvgradfill.obj
 0001:00017604       ?drvRectFill8@@YAXPAVGPESurf@@PAU_DRVGRADIENTRECTDATA@@@Z 10018604 f   gpe:rdrvgradfill.obj
 0001:00017618       ?drvRectFill4@@YAXPAVGPESurf@@PAU_DRVGRADIENTRECTDATA@@@Z 10018618 f   gpe:rdrvgradfill.obj
 0001:0001762c       ?drvRectFill1@@YAXPAVGPESurf@@PAU_DRVGRADIENTRECTDATA@@@Z 1001862c f   gpe:rdrvgradfill.obj
 0001:00017d24       DrvGradientFill            10018d24 f   gpe:rdrvgradfill.obj
 0001:0001858c       DrvAlphaBlend              1001958c f   gpe:drvalphablend.obj
 0001:00018614       GenBltInitialize           10019614 f   gpe:genblt.obj
 0001:000187cc       ?ClockOverflow@@YAXXZ      100197cc f   gpe:genblt.obj
 0001:0001880c       ?FunctionCacheLookup@@YAPAUGenBltFunction@@PAUGenBltSignature@@@Z 1001980c f   gpe:genblt.obj
 0001:00018878       ?GetFnCacheMem@@YAPAUGenBltFunction@@PAUGenBltSignature@@@Z 10019878 f   gpe:genblt.obj
 0001:000188f8       ?GetBltFunction@@YAPAUGenBltFunction@@PAUGenBltSignature@@@Z 100198f8 f   gpe:genblt.obj
 0001:000189ac       ?GPEFormatToGenBltFormat@@YA?AW4GenBltFormat@@PAVGPEFormat@@W4EGPEFormat@@@Z 100199ac f   gpe:genblt.obj
 0001:00018b24       GenBltSetMode              10019b24 f   gpe:genblt.obj
 0001:00018d30       ?GenerateSignature@@YAHPAUGPEBltParms@@PAUGenBltSignature@@@Z 10019d30 f   gpe:genblt.obj
 0001:000191bc       ?ProcessROP3@@YAKKKKEE@Z   1001a1bc f   gpe:BltHelpers.obj
 0001:0001927c       ?RGBError@@YAKKK@Z         1001a27c f   gpe:BltHelpers.obj
 0001:000192c0       ?FillMasksAndShifts@@YAXPAVGPESurf@@PAK1@Z 1001a2c0 f   gpe:BltHelpers.obj
 0001:00019330       ?ClipRect@@YA_NPAU_RECTL@@PBU1@1@Z 1001a330 f   gpe:BltHelpers.obj
 0001:000193b0       ?AveragePixels@@YAKKKHHPAK0@Z 1001a3b0 f   gpe:BltHelpers.obj
 0001:00019510       ?AverageAndClampPixels@@YAKKKHHPAK0@Z 1001a510 f   gpe:BltHelpers.obj
 0001:000196b4       ?HalftoneBlend16Bpp@@YAXPAEKHHPAK1@Z 1001a6b4 f   gpe:BltHelpers.obj
 0001:000196ec       ?HalftoneBlend24Bpp@@YAXPAEKHHPAK1@Z 1001a6ec f   gpe:BltHelpers.obj
 0001:00019740       ?HalftoneBlend32Bpp@@YAXPAEKHHPAK1@Z 1001a740 f   gpe:BltHelpers.obj
 0001:00019774       ?InitPixelIterator@PixelIterator@@QAAXPAVGPESurf@@HHPAU_RECTL@@HH@Z 1001a774 f   gpe:PixelIterator.obj
 0001:00019944       ?InitPixelIterator@PixelIteratorRotate@@QAAXPAVGPESurf@@HHPAU_RECTL@@HH@Z 1001a944 f   gpe:PixelIterator.obj
 0001:00019aa4       ?GetPtr@PixelIteratorRotate@@QAAPAEXZ 1001aaa4 f   gpe:PixelIterator.obj
 0001:00019b90       ?InitBrushPixelIterator@BrushPixelIterator@@QAAXPAVGPESurf@@HHPAU_RECTL@@@Z 1001ab90 f   gpe:PixelIterator.obj
 0001:00019c7c       ?WrappedGeneratedBlt@GPE@@QAAJPAUGPEBltParms@@@Z 1001ac7c f   gpe:GenBltGpe.obj
 0001:00019d7c       GeneratedBltSelect         1001ad7c f   gpe:GenBltGpe.obj
 0001:00019dcc       EmulatedBltSelect02        1001adcc f   gpe:ebbltsel.obj
 0001:00019dd4       EmulatedBltSelect08        1001add4 f   gpe:ebbltsel.obj
 0001:00019ffc       EmulatedBltSelect16        1001affc f   gpe:ebbltsel.obj
 0001:0001a1d0       ?IsSurface_R5_G6_B5@@YAHPAVGPESurf@@@Z 1001b1d0 f i gpe:FastBlt.obj
 0001:0001a228       ?IsSurface_A8_R8_G8_B8@@YAHPAVGPESurf@@@Z 1001b228 f i gpe:FastBlt.obj
 0001:0001a28c       ?CanUse_Blt_Stretch_Alpha_32To16at565@@YAHPAUGPEBltParms@@@Z 1001b28c f i gpe:FastBlt.obj
 0001:0001a388       ?Blt_Stretch_Alpha_32To16at565@Emulator@@QAAJPAUGPEBltParms@@@Z 1001b388 f   gpe:FastBlt.obj
 0001:0001ab24       ?CanUse_Blt_NoStretch_Alpha_32To16at565@@YAHPAUGPEBltParms@@@Z 1001bb24 f i gpe:FastBlt.obj
 0001:0001ab60       ?Blt_NoStretch_Alpha_32To16at565@Emulator@@QAAJPAUGPEBltParms@@@Z 1001bb60 f   gpe:FastBlt.obj
 0001:0001aeac       ?CanUse_Blt_NoStretch_Alpha_24To24@@YAHPAUGPEBltParms@@@Z 1001beac f i gpe:FastBlt.obj
 0001:0001af44       ?Blt_NoStretch_Alpha_24To24_Aligned@@YAJPAKH0HHHK@Z 1001bf44 f   gpe:FastBlt.obj
 0001:0001b088       ?Blt_NoStretch_Alpha_24To24@Emulator@@QAAJPAUGPEBltParms@@@Z 1001c088 f   gpe:FastBlt.obj
 0001:0001b260       ?CanUse_Blt_NoStretch_Alpha_16To16@@YAHPAUGPEBltParms@@@Z 1001c260 f i gpe:FastBlt.obj
 0001:0001b308       ?Blt_NoStretch_Alpha_16To16@Emulator@@QAAJPAUGPEBltParms@@@Z 1001c308 f   gpe:FastBlt.obj
 0001:0001b4e4       ?CanUse_Blt_NoStretch_Trans_16To16@@YAHPAUGPEBltParms@@@Z 1001c4e4 f i gpe:FastBlt.obj
 0001:0001b580       ?Blt_NoStretch_Trans_16To16@Emulator@@QAAJPAUGPEBltParms@@@Z 1001c580 f   gpe:FastBlt.obj
 0001:0001b648       ?CanUse_Blt_Stretch_Trans_16To16@@YAHPAUGPEBltParms@@@Z 1001c648 f i gpe:FastBlt.obj
 0001:0001b6e8       ?CanUse_Blt_NoStretch_NoTrans_32To16at565@@YAHPAUGPEBltParms@@@Z 1001c6e8 f i gpe:FastBlt.obj
 0001:0001b780       ?Blt_NoStretch_NoTrans_32To16at565@Emulator@@QAAJPAUGPEBltParms@@@Z 1001c780 f   gpe:FastBlt.obj
 0001:0001b84c       ?CanUse_Blt_NoStretch_NoTrans_16at565To32@@YAHPAUGPEBltParms@@@Z 1001c84c f i gpe:FastBlt.obj
 0001:0001b8f0       ?Blt_NoStretch_NoTrans_16at565To32@Emulator@@QAAJPAUGPEBltParms@@@Z 1001c8f0 f   gpe:FastBlt.obj
 0001:0001b9b8       ?CanUse_Blt_NoStretch_NoTrans_24To24@@YAHPAUGPEBltParms@@@Z 1001c9b8 f i gpe:FastBlt.obj
 0001:0001ba50       ?Blt_NoStretch_NoTrans_24To24@Emulator@@QAAJPAUGPEBltParms@@@Z 1001ca50 f   gpe:FastBlt.obj
 0001:0001bb08       ?CanUse_Blt_NoStretch_NoTrans_16To16@@YAHPAUGPEBltParms@@@Z 1001cb08 f i gpe:FastBlt.obj
 0001:0001bba0       ?Blt_NoStretch_NoTrans_16To16@Emulator@@QAAJPAUGPEBltParms@@@Z 1001cba0 f   gpe:FastBlt.obj
 0001:0001bc54       ?CanUse_Blt_Text_32@@YAHPAUGPEBltParms@@@Z 1001cc54 f i gpe:FastBlt.obj
 0001:0001bce0       ?Blt_Text_32@Emulator@@QAAJPAUGPEBltParms@@@Z 1001cce0 f   gpe:FastBlt.obj
 0001:0001bdd8       ?CanUse_Blt_Fill_32@@YAHPAUGPEBltParms@@@Z 1001cdd8 f i gpe:FastBlt.obj
 0001:0001be34       ?Blt_Fill_32@Emulator@@QAAJPAUGPEBltParms@@@Z 1001ce34 f   gpe:FastBlt.obj
 0001:0001becc       ?CanUse_Blt_Fill_24@@YAHPAUGPEBltParms@@@Z 1001cecc f i gpe:FastBlt.obj
 0001:0001bf28       ?Blt_Fill_24@Emulator@@QAAJPAUGPEBltParms@@@Z 1001cf28 f   gpe:FastBlt.obj
 0001:0001bfe0       ?Blt_Stretch_Trans_16To16@Emulator@@QAAJPAUGPEBltParms@@@Z 1001cfe0 f   gpe:FastBlt.obj
 0001:0001c680       FastBltSelect              1001d680 f   gpe:FastBlt.obj
 0001:0001c86c       GenBltCpuInitialize        1001d86c f   gpe:genblt_arm.obj
 0001:0001c898       ?RopRecurse@@YAFPAKF@Z     1001d898 f   gpe:parse.obj
 0001:0001c9b8       ?ConvertRecurse@@YAFPAKKF@Z 1001d9b8 f   gpe:parse.obj
 0001:0001cbb0       ?GenBltInvariantParser@@YA_NPAK0PAUGenBltSignature@@@Z 1001dbb0 f   gpe:parse.obj
 0001:0001ce9c       ?InvariantRecurse@@YAFPAKKKHF@Z 1001de9c f   gpe:parse.obj
 0001:0001d1e4       ?InvariantInitialize@@YAHPAK@Z 1001e1e4 f   gpe:parse.obj
 0001:0001d420       ?BRegFromBltSig@@YAKPAUGenBltSignature@@@Z 1001e420 f   gpe:InitRegs.obj
 0001:0001d574       ?InitPCodeRegs@@YAXPAUGPEBltParms@@PAUPCodeRegisters_t@@@Z 1001e574 f   gpe:InitRegs.obj
 0001:0001e2e8       ?EmulatedBltSrcCopy0108@Emulator@@QAAJPAUGPEBltParms@@@Z 1001f2e8 f   gpe:ebcp0108.obj
 0001:0001e75c       ?EmulatedBltSrcCopy0408@Emulator@@QAAJPAUGPEBltParms@@@Z 1001f75c f   gpe:ebcp0408.obj
 0001:0001e8e8       ?EmulatedBltSrcCopy0808@Emulator@@QAAJPAUGPEBltParms@@@Z 1001f8e8 f   gpe:ebcopy08.obj
 0001:0001ec68       ?EmulatedBltSrcPaint0808@Emulator@@QAAJPAUGPEBltParms@@@Z 1001fc68 f   gpe:ebspnt08.obj
 0001:0001f068       ?EmulatedBltPatternCopy08@Emulator@@QAAJPAUGPEBltParms@@@Z 10020068 f   gpe:ebpcpy08.obj
 0001:0001f444       ?EmulatedBltAlphaText08@Emulator@@QAAJPAUGPEBltParms@@@Z 10020444 f   gpe:ebalph08.obj
 0001:0001f464       ?EmulatedBltText08@Emulator@@QAAJPAUGPEBltParms@@@Z 10020464 f   gpe:ebtext08.obj
 0001:0001f5bc       ?EmulatedBltFill08@Emulator@@QAAJPAUGPEBltParms@@@Z 100205bc f   gpe:ebfill08.obj
 0001:0001f650       ?EmulatedBltDstInvert08@Emulator@@QAAJPAUGPEBltParms@@@Z 10020650 f   gpe:ebdinv08.obj
 0001:0001f758       ?EmulatedBltPatInvert08@Emulator@@QAAJPAUGPEBltParms@@@Z 10020758 f   gpe:ebpinv08.obj
 0001:0001f880       ?EmulatedBltPatternInvert08@Emulator@@QAAJPAUGPEBltParms@@@Z 10020880 f   gpe:ebp08.obj
 0001:0001fae4       ?EmulatedBltSrcInvert0808@Emulator@@QAAJPAUGPEBltParms@@@Z 10020ae4 f   gpe:ebsinv08.obj
 0001:0001fee4       ?EmulatedBltSrcAnd0808@Emulator@@QAAJPAUGPEBltParms@@@Z 10020ee4 f   gpe:ebsand08.obj
 0001:000202e4       ?EmulatedBltSrcPaint1616@Emulator@@QAAJPAUGPEBltParms@@@Z 100212e4 f   gpe:EBSPNT16.obj
 0001:000206e4       ?EmulatedBltSrcCopy0116@Emulator@@QAAJPAUGPEBltParms@@@Z 100216e4 f   gpe:ebcp0116.obj
 0001:00020b5c       ?EmulatedBltSrcCopy0416@Emulator@@QAAJPAUGPEBltParms@@@Z 10021b5c f   gpe:ebcp0416.obj
 0001:00020cec       ?EmulatedBltSrcCopy1616@Emulator@@QAAJPAUGPEBltParms@@@Z 10021cec f   gpe:EBCOPY16.obj
 0001:00021094       ?EmulatedBltFill16@Emulator@@QAAJPAUGPEBltParms@@@Z 10022094 f   gpe:ebfill16.obj
 0001:00021154       ?EmulatedBltSrcInvert1616@Emulator@@QAAJPAUGPEBltParms@@@Z 10022154 f   gpe:EBSINV16.obj
 0001:00021554       ?EmulatedBltSrcAnd1616@Emulator@@QAAJPAUGPEBltParms@@@Z 10022554 f   gpe:ebsand16.obj
 0001:00021954       ?EmulatedBltAlphaText16@Emulator@@QAAJPAUGPEBltParms@@@Z 10022954 f   gpe:ebalph16.obj
 0001:00021974       ?EmulatedBltText16@Emulator@@QAAJPAUGPEBltParms@@@Z 10022974 f   gpe:ebtext16.obj
 0001:00021acc       DDKGpioWriteDataPin        10022acc f   cspddk:CSPDDK.dll
 0001:00021adc       DDKGpioSetConfig           10022adc f   cspddk:CSPDDK.dll
 0001:00021aec       DDKIomuxSetPadConfig       10022aec f   cspddk:CSPDDK.dll
 0001:00021afc       DDKIomuxSetPinMux          10022afc f   cspddk:CSPDDK.dll
 0001:00021b0c       DDKClockSetGatingMode      10022b0c f   cspddk:CSPDDK.dll
 0001:00021b1c       DDKClockGetFreq            10022b1c f   cspddk:CSPDDK.dll
 0001:00021b2c       MmMapIoSpace               10022b2c f   ceddk:CEDDK.dll
 0001:00021b3c       MmUnmapIoSpace             10022b3c f   ceddk:CEDDK.dll
 0001:00021b4c       RegCloseKey                10022b4c f   coredll:COREDLL.dll
 0001:00021b5c       RegQueryValueExW           10022b5c f   coredll:COREDLL.dll
 0001:00021b6c       RegOpenKeyExW              10022b6c f   coredll:COREDLL.dll
 0001:00021b7c       RegSetValueExW             10022b7c f   coredll:COREDLL.dll
 0001:00021b8c       EventModify                10022b8c f   coredll:COREDLL.dll
 0001:00021b9c       VirtualSetAttributes       10022b9c f   coredll:COREDLL.dll
 0001:00021bac       VirtualCopy                10022bac f   coredll:COREDLL.dll
 0001:00021bbc       VirtualAlloc               10022bbc f   coredll:COREDLL.dll
 0001:00021bcc       AllocPhysMem               10022bcc f   coredll:COREDLL.dll
 0001:00021bdc       FreePhysMem                10022bdc f   coredll:COREDLL.dll
 0001:00021bec       VirtualFree                10022bec f   coredll:COREDLL.dll
 0001:00021bfc       Sleep                      10022bfc f   coredll:COREDLL.dll
 0001:00021c0c       DeleteCriticalSection      10022c0c f   coredll:COREDLL.dll
 0001:00021c1c       WaitForSingleObject        10022c1c f   coredll:COREDLL.dll
 0001:00021c2c       CloseHandle                10022c2c f   coredll:COREDLL.dll
 0001:00021c3c       KernelIoControl            10022c3c f   coredll:COREDLL.dll
 0001:00021c4c       InterruptDisable           10022c4c f   coredll:COREDLL.dll
 0001:00021c5c       InterruptDone              10022c5c f   coredll:COREDLL.dll
 0001:00021c6c       LeaveCriticalSection       10022c6c f   coredll:COREDLL.dll
 0001:00021c7c       EnterCriticalSection       10022c7c f   coredll:COREDLL.dll
 0001:00021c8c       ExitThread                 10022c8c f   coredll:COREDLL.dll
 0001:00021c9c       SystemParametersInfoW      10022c9c f   coredll:COREDLL.dll
 0001:00021cac       ChangeDisplaySettingsEx    10022cac f   coredll:COREDLL.dll
 0001:00021cbc       InitializeCriticalSection  10022cbc f   coredll:COREDLL.dll
 0001:00021ccc       CreateThread               10022ccc f   coredll:COREDLL.dll
 0001:00021cdc       InterruptInitialize        10022cdc f   coredll:COREDLL.dll
 0001:00021cec       CreateEventW               10022cec f   coredll:COREDLL.dll
 0001:00021cfc       WaitForMultipleObjects     10022cfc f   coredll:COREDLL.dll
 0001:00021d0c       TerminateThread            10022d0c f   coredll:COREDLL.dll
 0001:00021d1c       SetLastError               10022d1c f   coredll:COREDLL.dll
 0001:00021d2c       AdvertiseInterface         10022d2c f   coredll:COREDLL.dll
 0001:00021d3c       GetModuleFileNameW         10022d3c f   coredll:COREDLL.dll
 0001:00021d4c       GetCallerVMProcessId       10022d4c f   coredll:COREDLL.dll
 0001:00021d5c       RemoteLocalFree            10022d5c f   coredll:COREDLL.dll
 0001:00021d6c       RemoteLocalAlloc           10022d6c f   coredll:COREDLL.dll
 0001:00021d7c       MulDiv                     10022d7c f   coredll:COREDLL.dll
 0001:00021d8c       DisableThreadLibraryCalls  10022d8c f   coredll:COREDLL.dll
 0001:00021d9c       RegCreateKeyExW            10022d9c f   coredll:COREDLL.dll
 0001:00021dac       LocalAlloc                 10022dac f   coredll:COREDLL.dll
 0001:00021dbc       LocalFree                  10022dbc f   coredll:COREDLL.dll
 0001:00021dcc       LocalReAlloc               10022dcc f   coredll:COREDLL.dll
 0001:00021ddc       CeSetExtendedPdata         10022ddc f   coredll:COREDLL.dll
 0001:00021dec       CacheRangeFlush            10022dec f   coredll:COREDLL.dll
 0001:00021f00       _DllMainCRTStartup         10022f00 f   corelib0:pegdmain.obj
 0001:00021f30       __GSHandlerCheckCommon     10022f30 f   corelib0:gshandler.obj
 0001:00021f6c       __GSHandlerCheck           10022f6c f   corelib0:gshandler.obj
 0001:00021f90       __security_init_cookie     10022f90 f   corelib0:seccinit.obj
 0001:00021fec       __security_check_cookie    10022fec f   corelib0:armsecgs.obj
 0001:00022000       __gsfailure                10023000 f   corelib0:armsecgs.obj
 0001:00022140       _cexit                     10023140 f   corelib0:cexit.obj
 0001:0002215c       _initterm                  1002315c f   corelib0:crt0dat.obj
 0001:00022190       _cinit                     10023190 f   corelib0:crt0dat.obj
 0001:000221c4       memcpy                     100231c4 f   corelib1:COREDLL.dll
 0001:000221d4       wcslen                     100231d4 f   corelib1:COREDLL.dll
 0001:000221e4       mbstowcs                   100231e4 f   corelib1:COREDLL.dll
 0001:000221f4       memset                     100231f4 f   corelib1:COREDLL.dll
 0001:00022204       ??2@YAPAXI@Z               10023204 f   corelib1:COREDLL.dll
 0001:00022214       __itos                     10023214 f   corelib1:COREDLL.dll
 0001:00022224       __utos                     10023224 f   corelib1:COREDLL.dll
 0001:00022234       __muls                     10023234 f   corelib1:COREDLL.dll
 0001:00022244       __stou                     10023244 f   corelib1:COREDLL.dll
 0001:00022254       __rt_udiv                  10023254 f   corelib1:COREDLL.dll
 0001:00022264       __rt_sdiv                  10023264 f   corelib1:COREDLL.dll
 0001:00022274       free                       10023274 f   corelib1:COREDLL.dll
 0001:00022284       __adds                     10023284 f   corelib1:COREDLL.dll
 0001:00022294       malloc                     10023294 f   corelib1:COREDLL.dll
 0001:000222a4       ??3@YAXPAX@Z               100232a4 f   corelib1:COREDLL.dll
 0001:000222b4       swscanf                    100232b4 f   corelib1:COREDLL.dll
 0001:000222c4       __C_specific_handler       100232c4 f   corelib1:COREDLL.dll
 0001:000222d4       wcscpy                     100232d4 f   corelib1:COREDLL.dll
 0001:000222e4       _purecall                  100232e4 f   corelib1:COREDLL.dll
 0001:000222f4       memmove                    100232f4 f   corelib1:COREDLL.dll
 0001:00022304       _XcptFilter                10023304 f   corelib1:COREDLL.dll
 0001:00022314       __security_gen_cookie2     10023314 f   corelib1:COREDLL.dll
 0001:00022324       __report_gsfailure         10023324 f   corelib1:COREDLL.dll
 0001:00022334       buildDDHALInfo             10023334 f   lcdc_common_topaz_v1:halcaps.obj
 0001:00022488       ?HalCreateSurface@@YAKPAU_DDHAL_CREATESURFACEDATA@@@Z 10023488 f   lcdc_common_topaz_v1:halsurf.obj
 0001:00022560       ?HalFlip@@YAKPAU_DDHAL_FLIPDATA@@@Z 10023560 f   lcdc_common_topaz_v1:halsurf.obj
 0001:0002257c       ?HalGetBltStatus@@YAKPAU_DDHAL_GETBLTSTATUSDATA@@@Z 1002357c f   lcdc_common_topaz_v1:halsurf.obj
 0001:000225e8       ?HalUpdateOverlay@@YAKPAU_DDHAL_UPDATEOVERLAYDATA@@@Z 100235e8 f   lcdc_common_topaz_v1:halsurf.obj
 0001:00022604       ?HalSetOverlayPosition@@YAKPAU_DDHAL_SETOVERLAYPOSITIONDATA@@@Z 10023604 f   lcdc_common_topaz_v1:halsurf.obj
 0001:00022620       ?HalSetColorKey@@YAKPAU_DDHAL_SETCOLORKEYDATA@@@Z 10023620 f   lcdc_common_topaz_v1:halsurf.obj
 0001:00022688       ?HalGetDriverInfo@@YAKPAU_DDHAL_GETDRIVERINFODATA@@@Z 10023688 f   lcdc_common_topaz_v1:haldd.obj
 0001:000226a0       DDGPECanCreateSurface      100236a0 f   ddgpe:ddhsurf.obj
 0001:000226f0       DDGPECreateSurface         100236f0 f   ddgpe:ddhsurf.obj
 0001:00022b40       DDGPELock                  10023b40 f   ddgpe:ddhsurf.obj
 0001:00022c4c       DDGPEUnlock                10023c4c f   ddgpe:ddhsurf.obj
 0001:00022c5c       DDGPEDestroySurface        10023c5c f   ddgpe:ddhsurf.obj
 0001:00022c98       DDGPEGetFlipStatus         10023c98 f   ddgpe:ddhsurf.obj
 0001:00022d04       DDGPESetPalette            10023d04 f   ddgpe:ddhsurf.obj
 0001:00022d14       DDGPECreatePalette         10023d14 f   ddgpe:ddhpalette.obj
 0001:00022d24       DDGPEDestroyPalette        10023d24 f   ddgpe:ddhpalette.obj
 0001:00022d34       DDGPESetEntries            10023d34 f   ddgpe:ddhpalette.obj
 0001:00022d44       DDGPEWaitForVerticalBlank  10023d44 f   ddgpe:ddhdd.obj
 0001:00022e48       DDGPEGetPixelFormatFromSurfaceDesc 10023e48 f   ddgpe:ddhutil.obj
 0001:00022fac       InterlockedExchange        10023fac f   coredll:COREDLL.dll
 0001:00022fbc       TerminateProcess           10023fbc f   coredll:COREDLL.dll
 0001:00023090       __IMPORT_DESCRIPTOR_CSPDDK 10024090     cspddk:CSPDDK.dll
 0001:000230a4       __IMPORT_DESCRIPTOR_CEDDK  100240a4     ceddk:CEDDK.dll
 0001:000230b8       __IMPORT_DESCRIPTOR_COREDLL 100240b8     coredll:COREDLL.dll
 0001:000230cc       __NULL_IMPORT_DESCRIPTOR   100240cc     cspddk:CSPDDK.dll
 0002:00000000       __imp_MmMapIoSpace         10025000     ceddk:CEDDK.dll
 0002:00000004       __imp_MmUnmapIoSpace       10025004     ceddk:CEDDK.dll
 0002:00000008       \177CEDDK_NULL_THUNK_DATA  10025008     ceddk:CEDDK.dll
 0002:0000000c       __imp_InterlockedExchange  1002500c     coredll:COREDLL.dll
 0002:00000010       __imp___report_gsfailure   10025010     corelib1:COREDLL.dll
 0002:00000014       __imp___security_gen_cookie2 10025014     corelib1:COREDLL.dll
 0002:00000018       __imp_TerminateProcess     10025018     coredll:COREDLL.dll
 0002:0000001c       __imp_RemoteLocalAlloc     1002501c     coredll:COREDLL.dll
 0002:00000020       __imp_RegCloseKey          10025020     coredll:COREDLL.dll
 0002:00000024       __imp_RegQueryValueExW     10025024     coredll:COREDLL.dll
 0002:00000028       __imp_RegOpenKeyExW        10025028     coredll:COREDLL.dll
 0002:0000002c       __imp_RegSetValueExW       1002502c     coredll:COREDLL.dll
 0002:00000030       __imp_EventModify          10025030     coredll:COREDLL.dll
 0002:00000034       __imp_VirtualSetAttributes 10025034     coredll:COREDLL.dll
 0002:00000038       __imp_VirtualCopy          10025038     coredll:COREDLL.dll
 0002:0000003c       __imp_VirtualAlloc         1002503c     coredll:COREDLL.dll
 0002:00000040       __imp_AllocPhysMem         10025040     coredll:COREDLL.dll
 0002:00000044       __imp_FreePhysMem          10025044     coredll:COREDLL.dll
 0002:00000048       __imp_VirtualFree          10025048     coredll:COREDLL.dll
 0002:0000004c       __imp_Sleep                1002504c     coredll:COREDLL.dll
 0002:00000050       __imp_DeleteCriticalSection 10025050     coredll:COREDLL.dll
 0002:00000054       __imp_WaitForSingleObject  10025054     coredll:COREDLL.dll
 0002:00000058       __imp_CloseHandle          10025058     coredll:COREDLL.dll
 0002:0000005c       __imp_KernelIoControl      1002505c     coredll:COREDLL.dll
 0002:00000060       __imp_InterruptDisable     10025060     coredll:COREDLL.dll
 0002:00000064       __imp_InterruptDone        10025064     coredll:COREDLL.dll
 0002:00000068       __imp_LeaveCriticalSection 10025068     coredll:COREDLL.dll
 0002:0000006c       __imp_EnterCriticalSection 1002506c     coredll:COREDLL.dll
 0002:00000070       __imp_ExitThread           10025070     coredll:COREDLL.dll
 0002:00000074       __imp_SystemParametersInfoW 10025074     coredll:COREDLL.dll
 0002:00000078       __imp_ChangeDisplaySettingsEx 10025078     coredll:COREDLL.dll
 0002:0000007c       __imp_InitializeCriticalSection 1002507c     coredll:COREDLL.dll
 0002:00000080       __imp_CreateThread         10025080     coredll:COREDLL.dll
 0002:00000084       __imp_InterruptInitialize  10025084     coredll:COREDLL.dll
 0002:00000088       __imp_CreateEventW         10025088     coredll:COREDLL.dll
 0002:0000008c       __imp_WaitForMultipleObjects 1002508c     coredll:COREDLL.dll
 0002:00000090       __imp_TerminateThread      10025090     coredll:COREDLL.dll
 0002:00000094       __imp_SetLastError         10025094     coredll:COREDLL.dll
 0002:00000098       __imp_AdvertiseInterface   10025098     coredll:COREDLL.dll
 0002:0000009c       __imp_GetModuleFileNameW   1002509c     coredll:COREDLL.dll
 0002:000000a0       __imp_GetCallerVMProcessId 100250a0     coredll:COREDLL.dll
 0002:000000a4       __imp_RemoteLocalFree      100250a4     coredll:COREDLL.dll
 0002:000000a8       __imp_MulDiv               100250a8     coredll:COREDLL.dll
 0002:000000ac       __imp_DisableThreadLibraryCalls 100250ac     coredll:COREDLL.dll
 0002:000000b0       __imp_RegCreateKeyExW      100250b0     coredll:COREDLL.dll
 0002:000000b4       __imp_LocalAlloc           100250b4     coredll:COREDLL.dll
 0002:000000b8       __imp_LocalFree            100250b8     coredll:COREDLL.dll
 0002:000000bc       __imp_LocalReAlloc         100250bc     coredll:COREDLL.dll
 0002:000000c0       __imp_CeSetExtendedPdata   100250c0     coredll:COREDLL.dll
 0002:000000c4       __imp_CacheRangeFlush      100250c4     coredll:COREDLL.dll
 0002:000000c8       __imp_memcpy               100250c8     corelib1:COREDLL.dll
 0002:000000cc       __imp_wcslen               100250cc     corelib1:COREDLL.dll
 0002:000000d0       __imp_mbstowcs             100250d0     corelib1:COREDLL.dll
 0002:000000d4       __imp_memset               100250d4     corelib1:COREDLL.dll
 0002:000000d8       __imp_??2@YAPAXI@Z         100250d8     corelib1:COREDLL.dll
 0002:000000dc       __imp___itos               100250dc     corelib1:COREDLL.dll
 0002:000000e0       __imp___utos               100250e0     corelib1:COREDLL.dll
 0002:000000e4       __imp___muls               100250e4     corelib1:COREDLL.dll
 0002:000000e8       __imp___stou               100250e8     corelib1:COREDLL.dll
 0002:000000ec       __imp___rt_udiv            100250ec     corelib1:COREDLL.dll
 0002:000000f0       __imp___rt_sdiv            100250f0     corelib1:COREDLL.dll
 0002:000000f4       __imp_free                 100250f4     corelib1:COREDLL.dll
 0002:000000f8       __imp___adds               100250f8     corelib1:COREDLL.dll
 0002:000000fc       __imp_malloc               100250fc     corelib1:COREDLL.dll
 0002:00000100       __imp_??3@YAXPAX@Z         10025100     corelib1:COREDLL.dll
 0002:00000104       __imp_swscanf              10025104     corelib1:COREDLL.dll
 0002:00000108       __imp___C_specific_handler 10025108     corelib1:COREDLL.dll
 0002:0000010c       __imp_wcscpy               1002510c     corelib1:COREDLL.dll
 0002:00000110       __imp__purecall            10025110     corelib1:COREDLL.dll
 0002:00000114       __imp___divs               10025114     corelib1:COREDLL.dll
 0002:00000118       __imp___stod               10025118     corelib1:COREDLL.dll
 0002:0000011c       __imp_pow                  1002511c     corelib1:COREDLL.dll
 0002:00000120       __imp___dtos               10025120     corelib1:COREDLL.dll
 0002:00000124       __imp___subs               10025124     corelib1:COREDLL.dll
 0002:00000128       __imp___rt_sdiv64by64      10025128     corelib1:COREDLL.dll
 0002:0000012c       __imp_memmove              1002512c     corelib1:COREDLL.dll
 0002:00000130       __imp__XcptFilter          10025130     corelib1:COREDLL.dll
 0002:00000134       \177COREDLL_NULL_THUNK_DATA 10025134     coredll:COREDLL.dll
 0002:00000138       __imp_DDKClockGetFreq      10025138     cspddk:CSPDDK.dll
 0002:0000013c       __imp_DDKClockSetGatingMode 1002513c     cspddk:CSPDDK.dll
 0002:00000140       __imp_DDKIomuxSetPinMux    10025140     cspddk:CSPDDK.dll
 0002:00000144       __imp_DDKIomuxSetPadConfig 10025144     cspddk:CSPDDK.dll
 0002:00000148       __imp_DDKGpioSetConfig     10025148     cspddk:CSPDDK.dll
 0002:0000014c       __imp_DDKGpioWriteDataPin  1002514c     cspddk:CSPDDK.dll
 0002:00000150       \177CSPDDK_NULL_THUNK_DATA 10025150     cspddk:CSPDDK.dll
 0002:000001e0       ?_rgbIdentity@@3PAUtagPALETTEENTRY@@A 100251e0     lcdc_common_topaz_v1:DDLcdc.obj
 0002:000005e0       ?_rgb2bpp@@3PAUtagRGBQUAD@@A 100255e0     lcdc_common_topaz_v1:DDLcdc.obj
 0002:000005f0       ?_rgb4bpp@@3PAUtagRGBQUAD@@A 100255f0     lcdc_common_topaz_v1:DDLcdc.obj
 0002:0000069c       ?gaMix@@3PAEA              1002569c     gpe:ddi_if.obj
 0002:00000ae8       ?gulGamma@@3KA             10025ae8     gpe:rctblt.obj
 0002:00000aec       ?szGamma@@3PAGA            10025aec     gpe:rctblt.obj
 0002:00000b10       ?szGammaValue@@3PAGA       10025b10     gpe:rctblt.obj
 0002:00000b28       ?alAlpha@@3PAJA            10025b28     gpe:rctblt.obj
 0002:00000b48       ?ajGammaCT_10@@3PAEA       10025b48     gpe:rctblt.obj
 0002:00000c48       ?ajGammaCT_11@@3PAEA       10025c48     gpe:rctblt.obj
 0002:00000d48       ?ajGammaInvCT_11@@3PAEA    10025d48     gpe:rctblt.obj
 0002:00000e48       ?ajGammaCT_12@@3PAEA       10025e48     gpe:rctblt.obj
 0002:00000f48       ?ajGammaInvCT_12@@3PAEA    10025f48     gpe:rctblt.obj
 0002:00001048       ?ajGammaCT_13@@3PAEA       10026048     gpe:rctblt.obj
 0002:00001148       ?ajGammaInvCT_13@@3PAEA    10026148     gpe:rctblt.obj
 0002:00001248       ?ajGammaCT_14@@3PAEA       10026248     gpe:rctblt.obj
 0002:00001348       ?ajGammaInvCT_14@@3PAEA    10026348     gpe:rctblt.obj
 0002:00001448       ?ajGammaCT_15@@3PAEA       10026448     gpe:rctblt.obj
 0002:00001548       ?ajGammaInvCT_15@@3PAEA    10026548     gpe:rctblt.obj
 0002:00001648       ?ajGammaCT_16@@3PAEA       10026648     gpe:rctblt.obj
 0002:00001748       ?ajGammaInvCT_16@@3PAEA    10026748     gpe:rctblt.obj
 0002:00001848       ?ajGammaCT_17@@3PAEA       10026848     gpe:rctblt.obj
 0002:00001948       ?ajGammaInvCT_17@@3PAEA    10026948     gpe:rctblt.obj
 0002:00001a48       ?ajGammaCT_18@@3PAEA       10026a48     gpe:rctblt.obj
 0002:00001b48       ?ajGammaInvCT_18@@3PAEA    10026b48     gpe:rctblt.obj
 0002:00001c48       ?ajGammaCT_19@@3PAEA       10026c48     gpe:rctblt.obj
 0002:00001d48       ?ajGammaInvCT_19@@3PAEA    10026d48     gpe:rctblt.obj
 0002:00001e48       ?ajGammaCT_20@@3PAEA       10026e48     gpe:rctblt.obj
 0002:00001f48       ?ajGammaInvCT_20@@3PAEA    10026f48     gpe:rctblt.obj
 0002:00002048       ?ajGammaCT_21@@3PAEA       10027048     gpe:rctblt.obj
 0002:00002148       ?ajGammaInvCT_21@@3PAEA    10027148     gpe:rctblt.obj
 0002:00002248       ?ajGammaCT_22@@3PAEA       10027248     gpe:rctblt.obj
 0002:00002348       ?ajGammaInvCT_22@@3PAEA    10027348     gpe:rctblt.obj
 0002:00002448       ?gaOutTable@@3PAU_F_RGB@@A 10027448     gpe:rctblt.obj
 0002:00002618       ?pfnDrvGradientFill@@3P6AHPAU_SURFOBJ@@PAU_CLIPOBJ@@PAU_XLATEOBJ@@PAU_TRIVERTEX@@KPAXKPAU_RECTL@@PAU_POINTL@@K@ZA 10027618     gpe:rdrvgradfill.obj
 0002:00002620       ?gulDither32@@3PAKA        10027620     gpe:rdrvgradfill.obj
 0002:00002660       ?gDitherMatrix16x16Halftone@@3PAEA 10027660     gpe:rdrvgradfill.obj
 0002:00002760       ?gDitherMatrix16x16Default@@3PAEA 10027760     gpe:rdrvgradfill.obj
 0002:00002860       ?vTranslateIdentity@@3PAEA 10027860     gpe:rdrvgradfill.obj
 0002:00002960       ?DefaultSaturationTable@@3PAEA 10027960     gpe:rdrvgradfill.obj
 0002:00002ae0       ?Saturation16_5@@3PAEA     10027ae0     gpe:rdrvgradfill.obj
 0002:00002b20       ?Saturation16_6@@3PAEA     10027b20     gpe:rdrvgradfill.obj
 0002:00002ba0       ?pfnDrvAlphaBlend@@3P6AHPAU_SURFOBJ@@0PAU_CLIPOBJ@@PAU_XLATEOBJ@@PAU_RECTL@@3PAUtagBLENDOBJ@@@ZA 10027ba0     gpe:drvalphablend.obj
 0002:00002ba8       ?g_pdwAnyBltPCode@@3PAKA   10027ba8     gpe:genblt.obj
 0002:0000bdfc       __security_cookie          10030dfc     corelib0:seccinit.obj
 0002:0000be00       __security_cookie_complement 10030e00     corelib0:seccinit.obj
 0002:0000be08       ?FSLFourCC@@3PAKA          10030e08     lcdc_common_topaz_v1:halcaps.obj
 0002:0000be10       ?cbDDCallbacks@@3U_DDHAL_DDCALLBACKS@@A 10030e10     lcdc_common_topaz_v1:halcaps.obj
 0002:0000be2c       ?MiscellaneousCallbacks@@3U_DDHAL_DDMISCELLANEOUSCALLBACKS@@A 10030e2c     lcdc_common_topaz_v1:halcaps.obj
 0002:0000be3c       ?cbDDPaletteCallbacks@@3U_DDHAL_DDPALETTECALLBACKS@@A 10030e3c     lcdc_common_topaz_v1:halcaps.obj
 0002:0000be4c       ?cbDDSurfaceCallbacks@@3U_DDHAL_DDSURFACECALLBACKS@@A 10030e4c     lcdc_common_topaz_v1:halcaps.obj
 0002:0000be80       ?VideoPortCallbacks@@3U_DDHAL_DDVIDEOPORTCALLBACKS@@A 10030e80     lcdc_common_topaz_v1:halcaps.obj
 0002:0000bed4       PATHOBJ_vGetBounds         10030ed4     gpe:ddi_if.obj
 0002:0000bed8       PATHOBJ_bEnum              10030ed8     gpe:ddi_if.obj
 0002:0000bedc       PALOBJ_cGetColors          10030edc     gpe:ddi_if.obj
 0002:0000bee0       CLIPOBJ_bEnum              10030ee0     gpe:ddi_if.obj
 0002:0000bee4       EngGetPaletteFromPool      10030ee4     gpe:ddi_if.obj
 0002:0000bee8       EngAddPaletteToPool        10030ee8     gpe:ddi_if.obj
 0002:0000beec       BRUSHOBJ_pvAllocRbrush     10030eec     gpe:ddi_if.obj
 0002:0000bef0       BRUSHOBJ_pvGetRbrush       10030ef0     gpe:ddi_if.obj
 0002:0000bef4       CLIPOBJ_cEnumStart         10030ef4     gpe:ddi_if.obj
 0002:0000bef8       XLATEOBJ_cGetPalette       10030ef8     gpe:ddi_if.obj
 0002:0000befc       PATHOBJ_vEnumStart         10030efc     gpe:ddi_if.obj
 0002:0000bf00       EngCreatePalette           10030f00     gpe:ddi_if.obj
 0002:0000bf04       EngCreateDeviceSurface     10030f04     gpe:ddi_if.obj
 0002:0000bf08       EngDeleteSurface           10030f08     gpe:ddi_if.obj
 0002:0000bf0c       EngCreateDeviceBitmap      10030f0c     gpe:ddi_if.obj
 0002:0000bf10       EngReleasePooledPalette    10030f10     gpe:ddi_if.obj
 0002:0000bf14       pfnGetGPEPerCard           10030f14     gpe:ddi_if.obj
 0002:0000bf18       g_hmodDisplayDll           10030f18     gpe:ddi_if.obj
 0002:0000bf1c       ?g_pxlo@@3PAU_XLATEOBJ@@A  10030f1c     gpe:ddi_if.obj
 0002:0000bf30       ?gMaskedConverter@@3PAVMaskColorConverter@@A 10030f30     gpe:swconvrt.obj
 0002:0000c0c0       ?gLookupConverter@@3PAVLookupColorConverter@@A 100310c0     gpe:swconvrt.obj
 0002:0000d110       ?gMonoConverter@@3PAVMonoColorConverter@@A 10032110     gpe:swconvrt.obj
 0002:0000d138       ?gMaskedLRU@@3VLRU@@A      10032138     gpe:swconvrt.obj
 0002:0000d14c       ?gLookupLRU@@3VLRU@@A      1003214c     gpe:swconvrt.obj
 0002:0000d160       ?gMonoLRU@@3VLRU@@A        10032160     gpe:swconvrt.obj
 0002:0000d174       ?gGroupLRU@@3VLRU@@A       10032174     gpe:swconvrt.obj
 0002:0000d188       ?gGroupConverter@@3PAVGroupColorConverter@@A 10032188     gpe:swconvrt.obj
 0002:0000dff8       ?pfnGetAAMaskBits@@3P6AXPAK00@ZA 10032ff8     gpe:aablt.obj
 0002:0000e044       ?gbHateMmx@@3HA            10033044     gpe:rctblt.obj
 0002:0000e4b8       ?g_BltFnPData@@3U_xpdata@@A 100334b8     gpe:genblt.obj
 0002:0000e540       ?g_CpuFuncs@@3UGenBltCpuFuncs@@A 10033540     gpe:genblt.obj
 0002:0000e55c       ?g_pPCodeRegisters@@3PAUPCodeRegisters_t@@A 1003355c     gpe:genblt.obj
 0002:0000e560       ?g_BltClock@@3KA           10033560     gpe:genblt.obj
 0002:0000e564       ?g_fUseFastBlt@@3HA        10033564     gpe:FastBlt.obj
 0002:0000fd80       _exitflag                  10034d80     corelib0:cexit.obj
 0002:0000fd84       ?g_nVideoMemorySize@@3KA   10034d84     lcdc_common_topaz_v1:halcaps.obj
 0002:0000fd88       ?g_pVideoMemory@@3PAEA     10034d88     lcdc_common_topaz_v1:halcaps.obj
 0002:0000fd8c       __onexitend                10034d8c     <common>
 0002:0000fd90       __onexitbegin              10034d90     <common>
 0002:0000fd94       g_pcsExit                  10034d94     <common>
 0002:0000fd98       _pRawDllMain               10034d98     <common>

 entry point at        0001:00021f00

 Static symbols

 0001:00001838       ?TurnOnLCD@@YAHPAULCDC_MODE_DESCRIPTOR@@@Z 10002838 f   bsplcdc.obj
 0001:0000529c       ?FillHelCaps@@YAXPAU_DDCAPS@@@Z 1000629c f   ddgpe:ddhinit.obj
 0001:00006880       ?AASetFormat@@YAJPAUGPEBltParms@@PAU_SURFOBJ@@@Z 10007880 f   gpe:ddi_if.obj
 0001:00013650       ?GetAAMaskInfo@@YAXH@Z     10014650 f   gpe:aablt.obj
 0001:000137b0       ?InitGamma@@YAXXZ          100147b0 f   gpe:aablt.obj
 0001:00014120       ?GetNearestIndex@@YAKK@Z   10015120 f   gpe:rctblt.obj
 0001:00014b14       ?vGetBlendInfo@@YAXKKPAVGPESurf@@PAU_BLENDINFO@@@Z 10015b14 f   gpe:rctblt.obj
 0001:00015d78       ?MDiv64@@YA_J_J00@Z        10016d78 f   gpe:rdrvgradfill.obj
 0001:00017b18       ?RectFillBlt@@YAHPAU_SURFOBJ@@PAU_DRVGRADIENTRECTDATA@@P6AXPAVGPESurf@@1@Z@Z 10018b18 f   gpe:rdrvgradfill.obj
 0001:00017ce4       ?GFGetShift@@YAXKPAK0@Z    10018ce4 f   gpe:rdrvgradfill.obj
 0001:00021e04       _DllMainCRTStartupHelper   10022e04 f   corelib0:pegdmain.obj
 0001:00022044       doexit                     10023044 f   corelib0:cexit.obj
 0001:00022fcc       ??__EgGroupConverter@@YAXXZ 10023fcc f   gpe:swconvrt.obj
